:100000000200377DA37C08ED1D70011C144C70F7B5
:10001000EF1F70011E144E70EA228FCFD209200903
:02002000FD22BF
:100023000208CBEF700753CEEF53CE7F2243CE109F
:1000330043CE8022787FE4F6D8FD7581280206FC42
:07004300759500759600227F
:10004B00020916E518240CF8E60518227809300782
:10005B0002780CE475F00112055A0203AA2000EB9A
:10006B007F2ED2008018EF540F2490D43440D4FF4D
:10007B0030040BEF24BFB41A0050032461FFE519C1
:10008B0060021519051CE51C7002051B30070D7865
:10009B0009E475F00112055AEF0205120209B97451
:1000AB0003D2078003E4C207F5188B098A0A890B70
:1000BB00E4F519F51BF51CE51960077F2012008983
:1000CB0080F5751AFFC201C200C202C203C205C28B
:1000DB0006C208120057FF700D3007057F00120093
:1000EB009AAF1CAE1B22B4255FC2D5C204120057B7
:1000FB00FF24D0B40A00501A75F00A781930D505D0
:10010B0008B6FF0106C6A426F620D5047002D2035A
:10011B0080D924CFB41A00EF5004C2E5D2040202F6
:10012B009AD20180C6D20080C0D20280BCD2D580C8
:10013B00BAD20580B47F201200892002077401B562
:10014B00190040F112004EFF1200890200C2D208C2
:10015B00D206809512004EFB12004EFA12004EF999
:10016B004A4B7006796B7A037BFF20022EE51960F0
:10017B002A7E008E827583001203C360060EEE6525
:10018B001A70F0C2D5EBC0E0EAC0E0E9C0E0EE12B5
:10019B0002E1D0E0F9D0E0FAD0E0FB1203AAFF6055
:1001AB00AAEBC0E0EAC0E0E9C0E0120089D0E0248D
:1001BB0001F9D0E03400FAD0E0FBE51A0460DCD59D
:1001CB001AD980877BFF7A0279DDD202809C791065
:1001DB0080027908C206C2088008D2D5790A800449
:1001EB00790AC2D5E51A047002F51AE4FAFDFEFF8E
:1001FB0012004EFC7B0820011312004EFD7B1030C9
:10020B00000A12004EFE12004EFF7B20EC3382D50B
:10021B0092D55013C3E43000069FFFE49EFEE4200A
:10022B0001039DFDE49CFCE4CBF8C201EC700CCF08
:10023B00CECDCCE824F8F870F38017C3EF33FFEE84
:10024B0033FEED33FDEC33FCEB33FB994002FB0F3C
:10025B00D8E9EB300105F8D0E0C448B201C0E00AA0
:10026B00EC4D4E4F78207B0070C2EAB51A0040BCB3
:10027B00C0E01202E3D0F0D0E0200104C4C0E0C41F
:10028B00B201C0F0120072D0F0D5F0EB0200C21236
:10029B00056A015F5301D95801304C012C4201DD35
:1002AB004F01E54401E54901454301EB5501CF46BB
:1002BB0001CF4501CF47038B5001342D01382E015F
:1002CB005B2B013C2301592003742A00F4480000E6
:1002DB0001533F3F3F00790AA2D520031430050993
:1002EB00B910020404B9080104A2D520060250017A
:1002FB00042002689202B519005034C0E07F203010
:10030B0003197F30A20272067205500F12033AC214
:10031B0002C206C205C2087F30800F300503E9C058
:10032B00E0120089300503D0E0F9D0E0B519CC30EC
:10033B0005177F30B9100C1200897F583004077FE6
:10034B00788003B908031200893002057F2D020063
:10035B00897F202008F87F2B2006F322920280CF82
:10036B00286E756C6C2900D20112004E3001F8C258
:10037B0001781930D50108F60200F42D5043495885
:10038B0012004E2403B405004001E490038693123F
:10039B00007A743A12007AD2037519040201D9BBA0
:1003AB00010689828A83E0225002E722BBFE02E328
:1003BB002289828A83E49322BB010CE58229F58290
:1003CB00E5833AF583E0225006E92582F8E622BB65
:1003DB00FE06E92582F8E222E58229F582E5833AD9
:1003EB00F583E4932275F008758200EF2FFFEE334F
:1003FB00FECD33CDCC33CCC58233C5829BED9AEC8D
:10040B0099E58298400CF582EE9BFEED9AFDEC99F6
:10041B00FC0FD5F0D6E4CEFBE4CDFAE4CCF9A88200
:10042B0022B800C1B90059BA002DEC8BF084CFCEA5
:10043B00CDFCE5F0CBF97818EF2FFFEE33FEED3363
:10044B00FDEC33FCEB33FB10D703994004EB99FB2A
:10045B000FD8E5E4F9FA227818EF2FFFEE33FEED13
:10046B0033FDEC33FCC933C910D7059BE99A400720
:10047B00EC9BFCE99AF90FD8E0E4C9FAE4CCFB2237
:10048B0075F010EF2FFFEE33FEED33FDCC33CCC800
:10049B0033C810D7079BEC9AE899400AED9BFDEC0B
:1004AB009AFCE899F80FD5F0DAE4CDFBE4CCFAE44A
:1004BB00C8F922EB9FF5F0EA9E42F0E99D42F0E885
:1004CB009C45F022E8600FECC313FCED13FDEE131B
:1004DB00FEEF13FFD8F122BB010DE58229F582E572
:1004EB00833AF5830205315007E92582F80205248A
:1004FB00BBFE07E92582F802053DE58229F582E579
:10050B00833AF58302054ABB010689828A83F0226E
:10051B005002F722BBFE01F322E6FB08E6F908E6E0
:10052B00FA08E6CBF822E0F8A3E0F9A3E0FAA3E09F
:10053B00FB22E2FB08E2F908E2FA08E2CBF822E43C
:10054B0093F8740193F9740293FA740393FB22FAF0
:10055B00E6FB0808E6F925F0F618E6CA3AF622D0CB
:10056B0083D082F8E4937012740193700DA3A3935C
:10057B00F8740193F5828883E4737402936860EFD7
:10058B00A3A3A380DF8B128A138914EF640160038A
:10059B000206F9752201F523F524F525F526F52735
:1005AB00F528FFEFC3948074809480500F74802FD4
:1005BB00F582E43400F583E4F00F80E7E4FFEFC34A
:1005CB00948074809480500F74002FF582E4340073
:1005DB00F583E4F00F80E7AB12AA13A9141203AA58
:1005EB00FFE598543F4FF598EF64C06008EF644007
:1005FB0060030206A89000021204E27F007E607D79
:10060B00547C0012042C8F188E178D168C15E4FF5A
:10061B00FE7D01FCAB18AA17A916A815C31204BEC0
:10062B0040037FFF22C3E49518F518E49517F517DF
:10063B0074019516F516E49515F515AB12AA13A9C9
:10064B00149000011203C364027026538EEF438E85
:10065B0001538EF7438E04AF18AE17AD16AC157859
:10066B00081204CF8FD68518D753AFFB438E10805B
:10067B0066C28E538EFE5389BF5389CF438E40AFD4
:10068B0018AE17AD16AC1578081204CF8F8D8518E0
:10069B008BC2AB5389BF538FFDD28E803AAB12AA5C
:1006AB0013A9141203AAFF7E007014900008120302
:1006BB00C364017005438E20801D538EDF8018EFBD
:1006CB0064804E70129000081203C36401700543DE
:1006DB008780800353877FAB12AA13A9149000075E
:1006EB001203C37004C29C8002D29C7F00227FFF46
:1006FB002212004312098812095CD2AF7BFF7A09E0
:10070B0079BE1200B07F017E00120003D3E527945F
:10071B00007480948040141527E527700ED3E526CE
:10072B009400748094804003752801E52860343070
:10073B00A231C2A27F01120026E4F508E508C39599
:10074B0026501474002508F582E43400F583E0FF8D
:10075B0012001A050880E5D2A2E4FF120026E4F588
:10076B0026F528D3E51D9400748094804097151DC1
:10077B00E51D7091D3E51E940074809480401EE4B7
:10078B00F508E508C3951E501474002508F582E49E
:10079B003401F583E0FF1209AF050880E5E4F51E8F
:1007AB000207109000011203C36401700553CE7F42
:1007BB00800343CE801203AAC4333354C0FFE5CE6B
:1007CB0054BF4FF5CE9000021203C3C43354E0FF65
:1007DB00E5CE54DF4FF5CE9000031203C3C454F0A3
:1007EB00FFE5CE54EF4FF5CE9000041203C3333325
:1007FB003354F8FFE5CE54F74FF5CE9000051203B6
:10080B00C325E025E0FFE5CE54FB4FF5CE90000667
:10081B001203C3FFE5CE54FC4FF5CEE4F51DC20920
:10082B0022EFD3940174809480500BEF25E0FFE509
:10083B00AF54FD4FF5AFEDFF7E00D394037480945E
:10084B0080502DEF700653B6FD53B5FDEF64014E8E
:10085B00700653B6FD43B502EF64024E700643B605
:10086B000253B5FDEF64034E700643B60243B50267
:10087B007F0022EFFBD39401748094805009EB70BE
:10088B0004C2AC8002D2ACEDFF7E00D39403748023
:10089B0094805029EF700553B7EFC2BCEF64014E43
:1008AB00700553B7EFD2BCEF64024E700543B7101F
:1008BB00C2BCEF64034E700543B710D2BC7F00225D
:1008CB00C0E0C083C082C0D075D000C0073098286C
:1008DB00C298E5287022C3E52694807480948040EA
:1008EB0003752600AF26052674002FF582E434002D
:1008FB00F583E599F0752705309905C299752500A3
:10090B00D007D0D0D082D083D0E032C0E0C083C03B
:10091B0082C0D075D000C007E5CE30E404C2098098
:10092B0022C3E51E9480748094804003751E00AF33
:10093B001E051E74002FF582E43401F583E5CFF01C
:10094B00751D0575CDC0D007D0D0D082D083D0E037
:10095B0032750901750A01E4F50BF50CF50D750EF1
:10096B0001F50FFB7A0079091207AE7D037F0112A7
:10097B00082CE5A254F34404F5A2D2A22275094037
:10098B00750A01750E00750DC2750C01750B00759E
:10099B0010017B007A0079097F011205907D017FA0
:1009AB000102087E8F99752501E52570FC22AE07A3
:1009BB000209AF53544338205541525431D3EB53B2
:0D09CB005049CDB8B4ABB3CCD0F20D0A004A
:00000001FF
